:10000000D628FF3FFF3FFF3F920003088301930084
:10001000803081079E1F640011182220911829202A
:100020001E181C209F0B3428A00B3428A40B342846
:100030002508A4009E1434282508A4009F01A001CF
:100040001E10080004308606940B080006111110DB
:10005000080004308606940B0800A20B08000C3040
:10006000A2000611911008001308830012080B115A
:1000700009008200413443344334453453344F340F
:1000800000345234453453345434523449344E34A9
:100090004734493444344F340034503441345334B9
:1000A0004534003434342E345334553450345234BF
:1000B00020344E34DF345534733475346134723443
:1000C00069346F34003431342E344D344F34443479
:1000D000493446342E34203443344F344434493484
:1000E00047344F3400342A342034533465346C346C
:1000F0002E340034233420347E34433441344E349F
:10010000433445344C34413444344F340034323475
:100110002E344E34DF344434493447344934543473
:100120004F345334203400345234653470346934DD
:100130007434613400345B3433343434353436341D
:100140005D34003433342E344E34DF3449344E348D
:10015000543445344E3454344F3453342034003402
:100160005B3430342D3439345D34003435342E343E
:1001700043344F3444342034503452344F345434A4
:1001800045344734203400345434653463346C349B
:10019000653465342034003442344C344F345134A7
:1001A00055344534413444344F340034850186019C
:1001B000910194010C30A2009E01831685017830D4
:1001C000860008308100A0308B0083122630402347
:1001D000A6006622C822363C03191E17A301EF228F
:1001E0001F305723EF220130A50031238530102323
:1001F0003A303723C2301023413037231E1B5B298E
:100200009E10AD229E18F22895002A3C03190D2954
:100210001508233C03193829002978239E18F32850
:100220001E19F32806309D000030CE231E1A19290E
:10023000272986173123863010234D303723692331
:1002400003305F23861302305F236622F3283123B5
:10025000CF305723911401305F23A70BF32883304D
:100260001023CC303723283040235F236622F32825
:100270003123752359303723AD229E18F3281E19D8
:10028000F328A300363023020318562A3030A30285
:1002900003194C29261B562A0330A50078239E18E3
:1002A000F3281E19F32801309D002308F423CE23E0
:1002B0001E1A5B2927291E13662269233123633006
:1002C0003723A122AD229E18F3281E1D6229950016
:1002D0002A3C03197129230803199429312369231E
:1002E000F3283123752387307F239E18562A1E1941
:1002F0005E29C03010233A30792294303723CF3032
:1003000057239114C7307F239E18562A1E195E2941
:1003100001309D003A30CE231E1A8F29562A230819
:1003200078226A2269235E293123873037232430DB
:1003300040233423A122AD229E18F3281E1D9B29A1
:1003400095002A3C0319A529E12931238730372359
:10035000C03010239B303723AD229E18F3281E197E
:100360009429950030309502073015020318AC2906
:1003700003301502031CAC291508960024304623CF
:100380000630950095031508CD2115087822CD215A
:100390009508031DC22969235E29F423A100402387
:1003A0009700DD219800DD219900DD219A00DD21F3
:1003B0009B00DD219C00BB230800A10A21084023EB
:1003C00008003123A2303723273040233423A122D1
:1003D000AD229E18F3281E1DE82995002A3C03191A
:1003E000F229042AC03010237523B0303723AD2200
:1003F0009E18F3281E19E129960030309602273006
:10040000462366226923E129312352303723A12272
:10041000AD229E18F3281E1D082A95002A3C0319B8
:10042000122A3E2AC03010237523AD229E18F328CD
:100430001E19042A95003030950206301502031863
:10044000152A01301502031C152A0030CD2115088C
:100450007822950B2C2AA610950B2F2A2611950B86
:10046000322AA611950B352A2612950B382AA61288
:1004700026089600263046236923042A3123B63005
:1004800037234E30261B53300E23A122AD229E1857
:10049000F3281E1D462A95002A3C0319502A542A87
:1004A0004030A60661223E2A6923F3283123833097
:1004B00010237D303723CF305723911403305F232F
:1004C000F3282608960026304623080027304023CC
:1004D000A700080023088D0001308E008D0A8D0BC7
:1004E000722A742A8E0D6F2A0E08A6046122080053
:1004F000F4238E22230803197E2A08000630A61C46
:100500008E220C30261D8E221230A61D8E2218300F
:10051000261E8E221E30A61E8E2208008D00170871
:100520009C2218089C2219089C221A089C221B084D
:100530009C221C089C22080096000D0846238D0A68
:100540000800C030102373303723CD3010237A30A9
:10055000372308002A300E2308001E14C1229E18DB
:100560000800C822003E0319AF2A11141E118D0085
:10057000233C03191E150D082A3C03191E150D08EE
:100580000800EC22C822003E031DC22AEC2208000B
:10059000CD22061086100510080086140514861D4D
:1005A0003134061E3434861E3734061F2A340614AE
:1005B0008610861D3234061E3534861E3834061FDA
:1005C000303486140510861D3334061E3634861EDC
:1005D0003934061F23340034203057230800861096
:1005E0000610033085000A23053057230A2305230C
:1005F0000A230523023085000A230523283010230F
:100600000C3010230630102308001F308D008D0B96
:10061000072B080005160000051208008614112B90
:10062000861006108C000C0E0F3985000A230C086A
:100630000F3985000A231D23080083160F3085001B
:1006400083128610061405169E178519252B9E13F6
:100650000512051600008501061083168501831218
:100660000800013010230800303E0E2308009000DF
:100670003920003E031908000E23900A1008382B79
:1006800089008316081483120808080089001608D8
:10069000880083168B13081555308900AA3089000D
:1006A00088148B17081E522B0812831208008D0025
:1006B000FF308E008E0B5A2B8D0B582B0800A1009B
:1006C00004308F00FF3057238F0B622BA10B602B60
:1006D0000800CF305723FF30572311147F305723A2
:1006E00011147F30572311140800C4303723080039
:1006F00031238130102375236C303723C030102311
:10070000243040239D00AD229E1808001E190800C9
:100710009700AA229D03AD229E1808001E1908000A
:100720009800AA229D03AD229E1808001E190800F9
:100730009900AA229D0B9D2BB92BAD229E18080073
:100740001E1908009A00AA229D0BA72BB92BAD22D7
:100750009E1808001E1908009B00AA229D0BB12BB1
:10076000B92BAD229E1808001E1908009C00AA2271
:10077000B92BBB230800243040239D0002309D028A
:1007800030309D0BC42BCA2B9D0BC72BCB2B9D0B45
:10079000CD2BCC2B9A009B009C0008008D001E12D4
:1007A0009E15F1231702EE238D0AF1231802EE2382
:1007B0008D0AF1231902EE238D0AF1231A02EE238A
:1007C0008D0AF1231B02EE238D0AF1231C02EE2376
:1007D0008D0A9E191E169D0BD02B0800031D9E111D
:1007E00008000D08402308008D0003190034003074
:1007F000063E8D0BF82B0800FF3FFF3FFF3FFF3FFA
:084000000F000F000F000F007C
:02400E00F53F7C
:10420000300030003000300030003000300030002E
:10421000300030003000300030003000300030001E
:10422000300030003000300030003000300030000E
:1042300030003000300030003000300030003000FE
:1042400030003000300030000400000000000300A7
:104250003D00FF00FF00FF00FF00FF00FF00FF0028
:10426000FF00FF00FF00FF00FF00FF00FF00FF0056
:10427000FF00FF0030003000300030003000300020
:00000001FF
